:101800005AC08EC073C072C071C070C06FC06EC04D
:101810006DC06CC06BC06AC069C068C067C066C07C
:1018200065C064C063C0EC2DFD2DB7B6B0FCFDCF24
:1018300027BFE895B7B6B0FCFDCF21E1B7B6B6FC3F
:10184000F4CF0895FFFFFFFFFFFFFFFFFFFFFFFF44
:10185000FFFFFFFFFFFFFFFFFFFFFFFFFFFFFFFF98
:10186000FFFFFFFF0902120001010080320904009E
:1018700000000000000012011001FF000008C01667
:10188000DC050201010200010E0355005300420075
:101890006100730070001C037700770077002E0052
:1018A000660069007300630068006C002E0064002D
:1018B00065000403090411241FBECFE5D4E0DEBF98
:1018C000CDBF10E0A0E6B0E0E8EFFFE102C0059078
:1018D0000D92A836B107D9F710E0A8E6B0E001C034
:1018E0001D92AC39B107E1F774D184C389CFA82F19
:1018F000B92F80E090E041E050EA609530E009C007
:101900002D9182279795879510F084279527305E33
:10191000C8F36F5FA8F30895EADF8D939D93089550
:10192000CF93CFB7CF93DF93C395869BE9F7869B81
:101930000BC0869B09C0869B07C0869B05C0869B03
:1019400003C0869B01C089C06F93C0917F00DD27D3
:10195000CA57DF4F2F9365E5869B03C02F916F9188
:10196000E6CF0F931F934F9320E040E15F9300B3C6
:10197000047406FB27F93F9350E03BE039C0147430
:1019800040642F77012F5F5F1EC0406810B314744E
:101990002F7752501FC0406400B32F770474D1F1E9
:1019A0005F5F00C023C0406210B32F77147491F1C1
:1019B0005F5F00C025C004741027515012F45D5FB2
:1019C0000000115027952C3F10B3C8F6147401275E
:1019D000015027952C3FC8F64227499300B3047461
:1019E00010274F73115027952C3FA8F64695469522
:1019F00010B3147479F00127015027952C3F98F605
:101A00006B5A60F3315000B3B0F600C010E41ABF57
:101A1000002717C03B503195C31BD04010E41ABFBC
:101A20000881033CF9F00B34E9F020917D00198125
:101A3000110F1213EDCF093651F10D3211F0013EA5
:101A400039F7009384003F915F914F911F910F915F
:101A50002F916F91CAB7C6FD67CFDF91CF91CFBFEE
:101A6000CF91189520918400222369F31091820070
:101A7000112339F534303AF13093820020937E00FF
:101A800010917F003BE0311B30937F001CC0009120
:101A900082000130B4F40AE53091610034FD14C0D5
:101AA00000936100C2E7D0E013C0052710E000C03A
:101AB000000002BB1AC0052710E0221F1DC010E065
:101AC00021C04AE502C032ED432FC4E1D0E032E04C
:101AD00011B31464969A02B311BB54E420E865E391
:101AE00020FF052702BB279517951C3FF0F666954A
:101AF000B8F7B1F720FF052702BB279517951C3FC4
:101B0000D0F62795179517FF052700001C3F02BB4D
:101B1000B0F629913A9519F70B7B10918300110FBC
:101B2000C651D04002BB11F010937D0010E41ABFE3
:101B3000006411B31B7B402F4B7B54E05A95F1F7A7
:101B400002BB11BB42BB7FCFDC0113963C911397C4
:101B5000932F1496EC9114978E2F12962C91129726
:101B6000203331F4E370F0E0EE59FF4F80810895A7
:101B7000283529F4332351F4E1E0F0E00BC020359F
:101B800071F4332321F5E0E0F0E004C03830E9F4EB
:101B9000E3E0F0E089E080935700849108952032DB
:101BA00021F4FC01EE0FFF1F06C0283231F4FC01C6
:101BB000EE0FFF1F319684910895203A09F405C273
:101BC000203C29F415966C9108D280E0089580E0BD
:101BD000089511BA80E882BB14BE81E08BBF82E019
:101BE0008BBF8799E6C185B7826085BF8BB780645C
:101BF0008BBF8E9A80E131978040E9F78E98789478
:101C0000D0918200D350D7FD40C120917F008CE05D
:101C100090E0821B910946E8A42E40E0B42EA80E65
:101C2000B91E20917E002D3209F0C8C0D83009F0CD
:101C30002AC123EC209372002AE5209361001092C0
:101C40006800D5013C91432F407611962C91119755
:101C50004423C9F189E690E090938100809380004D
:101C6000233031F4C50170DF80936C00C4E097C06D
:101C7000253039F12A3029F1822F84508630B0F492
:101C8000F5018281938190936E0080936D002930DD
:101C9000B1F0C681C0936F0085818270809370001F
:101CA0002093710037FD77C0CFEF75C08091600041
:101CB000223011F48E7F01C0816080936000C0E00B
:101CC0006EC0C1E06CC0D50112963C911297109283
:101CD0007B00222331F410927C008BE790E0C2E07D
:101CE00055C0253019F43093830044C02630E1F507
:101CF000FC01E857FF4F208187579F4FFC018081EF
:101D0000813019F486E798E104C0823041F484E61A
:101D100098E19093810080938000C2E121C08330DC
:101D2000F1F4222341F482EB98E1909381008093B7
:101D30008000C4E015C0213041F486E998E1909319
:101D4000810080938000CCE10BC0223041F488E810
:101D500098E19093810080938000CEE001C0C0E0C4
:101D600080E4809368001BC0283069F0293029F492
:101D7000309385008BE790E004C08BE790E02A3039
:101D800021F0C0E003C085E890E0C1E090938100BD
:101D90008093800004C080E8809368000CC0D50167
:101DA00017968C911797882331F416968C91169775
:101DB0008C1708F4C82FC093660065C08091680036
:101DC00087FF61C080916F008D1708F4D82F8D1B9D
:101DD00080936F0001E0811100E0809171008730F5
:101DE000B0F075010FC020916D0030916E00C901F7
:101DF000019690936E0080936D00F70161917F01D1
:101E0000C901EBD08E2D8A198D1768F338C08091E7
:101E10007000E0916D00F0916E00D501D0FDD3957A
:101E2000D25048F1F83138F522D0F8940D901D9039
:101E300021E017D02E2F2E5F2F7331F0002379F081
:101E4000882369F0D03059F423E00BD010D025E07E
:101E500008D00DD007B606FE02C021E102D03296AE
:101E6000DFCFF89427BFE89511247894089507B63A
:101E700000FCFDCF0895F0936E00E0936D00002309
:101E800011F010926600109282008091610084FF30
:101E900074C0809166008F3F09F46FC0D82F8930DD
:101EA00008F0D8E08D1B809366008091720098E85E
:101EB000892780937200DD2309F44EC08091680069
:101EC00087FF2AC080916F008D1708F4D82F8D1BD3
:101ED00080936F00DD2403E710E01BC08091710048
:101EE000E0906D00F0906E00873028F0C7016DD053
:101EF000F801808304C0F7018491D8018C930F5FAF
:101F00001F4F0894E11CF11CF0926E00E0926D00EE
:101F1000D394DD1619F71EC0E0918000F091810086
:101F200086FF09C08D2FA3E7B0E094919D93319671
:101F30008150D9F70BC0DF012D2F83E790E03D9151
:101F4000FC013193CF01FD012150C9F7F0938100CD
:101F5000E0938000D93058F483E790E06D2FDCDC0B
:101F6000DC5FDC3041F08FEF8093660004C08FEFC0
:101F700080936600DEE1D093610084E190B39474B5
:101F800031F48150D9F71092830010927D00809136
:101F90006000803118F08799805104C0823010F0C1
:101FA000879B82508093600080916000882309F0B5
:101FB00027CEF894EE278E9A9798EBBFE5BFF1E015
:101FC000FBBFEBBFFF270995EACEE199FECF9FBB90
:101FD0008EBBE09A99278DB30895262FE199FECF05
:101FE0009FBB8EBB2DBB0FB6F894E29AE19A0FBE51
:081FF00001960895F894FFCF5B
:081FF800FE5A1E930700FF00D2
:0400000300001800E1
:00000001FF
